:020000001C2AB8
:08000800FF00030E8312031335
:10001000B4000A0EB500040EB6008A110A12442A72
:10002000D508031D14280800F930FF3E031D1528CC
:100030000000D50B14280800E401E201E301600888
:10004000E500E601E4190800611C2C286508E207B8
:100050000318E30A6608E307E10C0310E50DE60D5B
:10006000E40A2228DD01DF01DE01DE1908000310A9
:10007000DF0DDB0DDD0D5C085D02031C4128DD009A
:100080005F14DE0A352883120313B908BA08B90AC7
:100090000319BA0A3B083906BC1B5A28031D5A2803
:1000A0003C083A06031D5A28480AC800B901BA019B
:1000B000470AC70048083B3C03187428520AD2007C
:1000C000C8014808DB000A30DC0032205F08D0009D
:1000D0005008E0000A30E1001C206208D9006308E3
:1000E000DA0059084802D10052083B3C03187D2829
:1000F0004E0ACE003C305202D2004E08173C031884
:10010000080018304E02CE00080004308316031396
:1001100009048900043083120905D500C6010430A2
:1001200055020319C60AC6080319AB28C6080319E5
:10013000A9280430831609048900043083120905B4
:10014000D500D601043055020319D60A5608C60058
:100150009628490AC9000130831609048900013034
:1001600083120905D500D30155030319D30AD30817
:100170000319D4285303031DCC2801308316090426
:100180008900013083120905D500D60155030319F2
:10019000D60A5608D300BA28540AD400FF30D50036
:1001A00010202D30D500102002308316090489005C
:1001B000023083120905D500CF0102305502031920
:1001C000CF0A5408013A0319EC28033A0319F82816
:1001D000013A0319042908004F03031D0800520ABD
:1001E000D200FF30D50010202D30D500102008009F
:1001F0004F03031D08004E0ACE00FF30D50010202B
:100200002D30D50010200800D401C8010800831249
:1002100003134808DB000A30DC0032205F08D000FE
:100220005008E0000A30E1001C206208D500630895
:10023000D60055084802D1005208DB000A30DC0025
:1002400032205F08CA004A08E0000A30E1001C20A2
:100250006208D5006308D60055085202CB00500E44
:10026000F039D0004903031D6E2904305007D00037
:10027000D1010430D000CB01CD01D6013908003CBA
:100280003A08BA1B46290318031DD60AD5010130C6
:100290003A02031D4D29F4303902031C5129BA1FBB
:1002A0005229D50A55085605031959291030510706
:1002B000D1008316850183125108850083168701BA
:1002C0008312500887008316860183124B0886002C
:1002D0008316880183124D0888000800D60139086A
:1002E000003C3A08BA1B77290318031DD60AD5012A
:1002F00001303A02031D7E29F4303902031C8229A1
:10030000BA1F8329D50A5508560503198A29903042
:100310005107D10008305007D0005208DB000A30E6
:10032000DC0032205F08CA004A08E0000A30E10021
:100330001C206208D7006308D80057085202CB007F
:100340004E08DB000A30DC0032205F08CC004C088D
:10035000E0000A30E1001C206208D7006308D800E2
:1003600057084E02CD004A0EF039CA004C0EF03943
:10037000CC008316850183125108850083168701FE
:10038000831250088700F030831606058600F0308F
:1003900083120605D7000F304B05570486000F3037
:1003A0008316060586000F3083120605D700F0304D
:1003B0004A0557048600F030831608058800F0309F
:1003C00083120805D7000F304D05570488000F3001
:1003D0008316080588000F3083120805D700F03017
:1003E0004C05570488004908013C031CC90108005A
:1003F0008316031788018901C03003138100E83098
:100400008312BB000330BC00C801CE01D201D4016D
:10041000B901BA010B17121092101215073012050C
:10042000D500183055049200F930831692008B17CE
:100430008C1485200721192AD53083120313A000BC
:10044000C430A100BB30A200DC30A300A401A50190
:10045000A601A701A801A901AA01AB01AC01AD0148
:10046000AE01AF01C001C101B701B801C201C301B2
:10047000C401C501B001B101B201B301BE01BF01A8
:10048000BD018A110A12F829831203138C1C4D2A0C
:1004900083168C1C4D2A43208C108312360E840048
:0E04A000350E8A00340E8300FF0E7F0E090019
:02400E00F2239B
:02401000FF3877
:00000001FF
